:020000040000FA
:02000000452891
:08000800F000030EF100831269
:1000100003138B1C0D28AB278B100B1C11281620EB
:0C0020000B10710E8300F00E700E090032
:1000400053298207563432342E343034313400345C
:100050008207413450344334003482074C344434F2
:10006000233423345034473453344D3450344334E0
:100070004334820744344C3447345034493449348F
:100080005334443454344334503485019701831637
:1000900006309F00F13085006130860081136030AA
:1000A0008F000F1D512883127A216122712286153B
:1000B0000530B100E822B10B5A288611B522061F7F
:1000C00087289B27831203135021051100008511F7
:1000D000FF30B400FA30B300061F872883120317DD
:1000E00063187E29831203130830B100B10B762800
:1000F000B30B6C2834081E3C031D7F28851434087C
:10010000013C031D84288510B40B6A286828A527A4
:10011000831203132708003C031D8F28F028D420E6
:100120004C211E30B400FF30B300E630B100301C6B
:100130009A28AF28061F9D286128B10B97283308FD
:10014000193C031DA42885143308013C031DA9286C
:100150008510B30B9528B40B9328DF2091285021EC
:10016000CC202108B100003E0319BB28061B6128E2
:10017000E822B10BB628851405152608B400003E08
:100180000319C928061FC62805116128EB22B40BE4
:10019000C228051185106E298515E82285110800F1
:1001A0000515E8220511080085152808B400003E51
:1001B0000319DD28E822B40BDA2885110800290884
:1001C000B400003E0319EF28CC202A08B300003EFB
:1001D0000319ED28E822B30BEA28B40BE428080041
:1001E000D4204C211E30B400FF30B300E630B10003
:1001F000301CFB281029061FFE286128B10BF828A7
:100200003308193C031D052985143308013C031DDF
:100210000A298510B30BF628B40BF428DF20F22846
:10022000502185102108B100003E03191C29061B2E
:100230006128E822B10B17292208B100003E0319FA
:1002400049292308B300003E03193B29061B6128F6
:1002500060213308013C031D2E293B292608240276
:10026000031C3929B400003E03193929E822B40BD4
:100270003629B30B26293108013C031847292508E4
:10028000B300003E03194729EB22B30B4429B10BFD
:100290002129E822E8226E2930108B158B170800DF
:1002A00030148B11080085102008B500003E03199A
:1002B0005E29861A0800D622B50B59293014080089
:1002C000051585142608B400003E03196B29E822A1
:1002D000E822B40B67290511851008005021EB2294
:1002E000061B78298B138B150B1063008B1170295B
:1002F000EB226128F522831203130800C82783121A
:1003000003132F3A031D86298F298E292F3A0D3A80
:10031000031D8D297A21E6298E290D3A612808309E
:10032000B300FA30B100831203176318A5298312B2
:100330000313D022B10B9329B30B91295430CD274D
:100340004F30CD27831203136128C827831203136C
:10035000523A031DAD291C2ADF29523A4E3A031D99
:10036000B3293D2ADF294E3A443A031DB929ED2924
:10037000DF29443A503A031DBF29FB29DF29503AAF
:100380004D3A031DC5295E2ADF294D3A563A031D11
:10039000CB296E2ADF29563A423A031DD229851409
:1003A000002FDF29423A533A031DD829812ADF2939
:1003B000533A5A3A031DDE297E2ADF295A3A45303C
:1003C000CD275230CD278312031361284F30CD271C
:1003D0004B30CD278312031361288514203084000D
:1003E0001030B1000008CD2783120313840AB10B2B
:1003F000F2298510E6298514A022203084001030CF
:10040000B300B830B1000C30B20083120317631888
:10041000122A83120313CB22B10B052AB20B052A31
:10042000B5229E29C827831203138000840AB30BC8
:10043000012AA0228510E6298514203084007A2123
:100440000030B100242AB10A31080A3C031C2F2ACB
:10045000310831220008FA227A21840A232A8510E1
:10046000E6292D20CD278312031331083920CD270B
:100470002D30CD278312031308008514A0222030CD
:1004800084000030B100452AB10A31080A3C031C3F
:100490005A2A7A213108312200082C2383120313AF
:1004A00080000008FF3C031D582AB5227A21E62966
:1004B000840A442A7A218510A022E6297A21612221
:1004C000E629B10131082820FF3903196C2ACD270C
:1004D00083120313B10A622A7A2108007A21712259
:1004E000E629B10131082120FF3903197C2ACD27E3
:1004F00083120313B10A722A7A2108001030CD2723
:10050000E6296021E629831203178C00831603175E
:100510008C130C158B1355308D00AA308D008C1464
:100520008C18902A8B178312031308008316031765
:100530008C130C14831203170C0883120313080086
:10054000203084000030B400A62AB40A34080F3CDE
:10055000031CB42A3408831203178D00831203137B
:1005600000088322840AA52A080083122030840010
:100570000030B400BC2AB40A34080F3C031CCA2A59
:100580003408831203178D00831203139622800010
:10059000840ABB2A0800A530F200F20BCD2A08001D
:1005A000C730F200D32AF20BD22A08002A30F20018
:1005B0004E30F300F30BDA2AF20BD82A080063302E
:1005C000F200A730F300F30BE32AF20BE12A080054
:1005D000DF22DF2208000A30F400E822F40BED2AC3
:1005E0000800CD278312031308000D30F1220A30D2
:1005F000F1220800F500F6016430F502031C022B1D
:10060000F60AFC2A6430F5077608003C0319182B1B
:100610007608303EF122F6010A30F502031C122B57
:10062000F60A0C2B0A30F5077608303EF122282B0B
:10063000F6010A30F502031C1F2BF60A192B0A30AB
:10064000F5077608003C0319282B7608303EF12286
:100650007508303EF1220800F700FF30FA226223CD
:100660007708FA227708633C031C382B2030F122EC
:100670007708093C031C3E2B2030F122C42783124B
:1006800003132B3A031D462BF70A602B2B3A2D3A06
:10069000031D4C2BF703602B2D3A303A031D522BD0
:1006A000F701602B303A1B3A031D582BFF34602BA7
:1006B0001B3A0D3A031D5F2B77080800602B0D3A9B
:1006C0002F2B08000830CD270830CD270830CD2744
:0206D000080020
:100E00009B2783120317E6014B30CD27C427523AA4
:100E1000031D0E2F2C2724274527232F523A573AFC
:100E2000031D192F2C275C272427342768277027B8
:100E3000232F573A453A031D222F2C2724273427E6
:100E40006827232F453A012FC427660203192B2F49
:100E50004330CD27002F0800C427E0398D00E60776
:100E6000C4278F00E60708000F08003C031D3D2F34
:100E70000D081F3C031C3D2F422F0F08063C031C8E
:100E8000422F08005230CD27002FE6012030E0002D
:100E9000831603178C170C1400000000831203172D
:100EA0000C08E607CD270E08E607CD278D0AE00BD4
:100EB000482F6608CD270800203084008317403073
:100EC000E000C427E6078000840AE00B612F0800D9
:100ED000831603178C170C168D2783120313080033
:100EE000831603178C170C1220308400831783128B
:100EF00003172030E0008312031700088C00840AD7
:100F000000088E00840A8D27831203178D0AE00BD8
:100F10007B2F8313831203130800831603170C150A
:100F20008B1355308D00AA308D008C14000000000A
:100F30008B170C11080083120317E101E3018316DC
:100F4000031301170B168B1708000B120800E4009F
:100F5000E40BA82F0800831203176310E314E201C7
:100F6000CB30A7270830E500061C03140618031031
:100F70008730A727E20CE50BB42F0618C32F6208B1
:100F8000E1006314E310080083120317631CC62FEB
:100F90008312031761086310080083120317E2002D
:100FA0008B1303100930E500031C86140318861008
:100FB0008730A727E20CE50BD42F86108930A727AE
:040FC0008B17080083
:02400E00103F61
:104200001400000001000C00100005000300000075
:104210000500050003000000000000000000000091
:00000001FF
